:020000040800F2
:1000000000000220D9040008D5070008D70700081F
:10001000D9070008DB070008DD0700080000000022
:10002000000000000000000000000000DF070008E2
:10003000E107000800000000E3070008E5070008EA
:1000400029050008290500082905000829050008D8
:100050002905000829050008ED0700082905000802
:1000600029050008290500082905000829050008B8
:1000700029050008290500082905000829050008A8
:1000800029050008290500082905000800000000CE
:10009000000000000000000000000000290500082A
:1000A00029050008F90700082905000829050008A6
:1000B0002905000829050008290500082905000868
:1000C0002905000829050008290500082905000858
:1000D000290500082905000829050008000000007E
:1000E000290500082905000829050008000000006E
:1000F00000000000000000000000000029050008CA
:10010000000000002905000829050008290500084D
:1001100000000000000000000000000000000000DF
:1001200029050008290500082905000829050008F7
:100130002905000800000000000000000000000089
:100140000000000000000000000000002905000879
:1001500029050008290500082905000829050008C7
:100160002905000829050008000000000000000023
:10017000000000000000000000000000000000007F
:100180000000000029050008000000000000000039
:080190002905000829050008FB
:1001980010B5054C237833B9044B13B10448AFF3B9
:1001A80000800123237010BD0C0000200000000017
:1001B8007814000808B5034B1BB103490348AFF393
:1001C800008008BD0000000010000020781400081E
:1001D80053B94AB9002908BF00281CBF4FF0FF31A6
:1001E8004FF0FF3000F072B9ADF1080C6DE904CEA4
:1001F80000F006F8DDF804E0DDE9022304B07047FA
:100208002DE9F047089E04468846002B4BD18A42C8
:10021800154667D9B2FA82F24AB1C2F1200701FA4B
:1002280002F320FA07F7954047EA030894404FEA9B
:10023800154E230CB8FBFEF71FFA85FC0EFB17883A
:1002480043EA084307FB0CF1994209D9EB1807F177
:10025800FF3080F01B81994240F21881023F2B4405
:100268005B1AA4B2B3FBFEF00EFB103344EA03445E
:1002780000FB0CFCA44509D92C1900F1FF3380F0D0
:100288000781A44540F2048102382C4440EA074023
:10029800A4EB0C0400271EB1D4400023C6E9004398
:1002A8003946BDE8F0878B4209D9002E00F0EB8073
:1002B8000027C6E9000138463946BDE8F087B3FA99
:1002C80083F7002F47D18B4202D3824200F2FA8093
:1002D800841A61EB030301209846002EE0D0C6E99A
:1002E8000048DDE702B9FFDEB2FA82F2002A40F0E8
:1002F8008F80491B4FEA154E1FFA85F80127B1FB7D
:10030800FEFC230C0EFB1C1143EA014308FB0CF115
:10031800994207D9EB180CF1FF3002D2994200F24A
:10032800CD808446591AA3B2B1FBFEF00EFB10141F
:1003380043EA044408FB00F8A04507D92C1900F14A
:10034800FF3302D2A04500F2B6801846A4EB080499
:1003580040EA0C409FE7C7F1200CBB4022FA0CFE94
:100368004EEA030E01FA07F420FA0CF521FA0CF311
:100378004FEA1E482543B3FBF8F92C0C08FB193348
:100388001FFA8EFA44EA034309FB0AF49C4202FA74
:1003980007F200FA07F10BD91EEB030309F1FF304E
:1003A80080F087809C4240F28480A9F1020973445E
:1003B8001B1BADB2B3FBF8F008FB103345EA03444E
:1003C80000FB0AFAA24508D91EEB040400F1FF332A
:1003D8006BD2A24569D90238744440EA0940A0FBAF
:1003E8000289A4EB0A044C45C2464B4654D351D06B
:1003F800002E69D0B1EB0A0564EB030404FA0CFC87
:10040800FD40FC404CEA0505C6E90054002747E7D3
:10041800C2F1200320FA03F7954001FA02F021FA0D
:1004280003F34FEA154E3843010CB3FBFEF71FFAEE
:1004380085F80EFB173341EA034107FB08F38B42AB
:1004480004FA02F407D9691807F1FF3C2FD28B424E
:100458002DD9023F2944CB1A81B2B3FBFEF00EFB23
:10046800103341EA034100FB08F38B4207D96918AE
:1004780000F1FF3C17D28B4215D902382944C91A1A
:1004880040EA07473BE73746304609E70746E7E6CD
:100498001846FBE64145ABD2B8EB020A69EB0E02FF
:1004A80001381346A4E76046E9E7184695E767462A
:1004B800D1E781467CE702382C4447E7ACF1020CCF
:1004C8002B442FE7384608E73746E9E6704700BF70
:1004D800DFF834D0002103E00C4B5B584350043163
:1004E8000B480C4B42189A42F6D30B4A02E0002301
:1004F80042F8043B094B9A42F9D300F081F900F025
:100508008BFF00F01DF9704700000220B8140008A6
:10051800000000200C0000200C00002070000020CB
:10052800FEE7000070B588B0002403940494059495
:10053800069407940094214B1A6B42F080021A63C8
:100548001A6B02F080020092009A01941A6B42F032
:1005580001021A631A6B02F001020192019A0294D5
:100568001A6B42F008021A631B6B03F0080302932C
:10057800029B134D22464FF47041284600F0F9FAC9
:10058800012603960F4B0493059403A90E4800F027
:1005980017FA4FF47043039304960594069403A93D
:1005A800284600F00DFA22462146062000F0B0F950
:1005B800062000F0E1F908B070BD00BF0038024025
:1005C800000C0240000011100000024008B5084865
:1005D800084B036042F20F7343600023836041F2CB
:1005E8008732C2600361836100F0FAFE08BD00BF74
:1005F8002C00002000440140012800D0704708B5B5
:100608000121064800F0AEFA012800D008BD0448D0
:1006180000F0B0FD034B01221A70F7E7000002401A
:100628002C0000202800002008B51E4B1B78012B49
:1006380000D008BD1B4B5B789BB1042B11D0012B5C
:1006480023D0052B21D0022B25D0062B23D0032B1A
:1006580001D0072B0AD14FF48041134800F08FFADC
:1006680004E04FF40041104800F089FA0D4A53782D
:100678000133DBB25370082BDBD1134600225A70CA
:100688001A700A4800F087FDD3E74FF480510648F6
:1006980000F075FAEAE74FF40051034800F06FFAEA
:1006A800E4E700BF28000020000C02402C000020D6
:1006B80030B595B03022002108A800F0D1FE002402
:1006C8000394049405940694079401941A4B1A6CA5
:1006D80042F080521A641B6C03F080530193019B13
:1006E8000294164B1A6842F440421A601B6803F4DD
:1006F80040430293029B012308934FF480330993EC
:1007080002250E954FF480030F930423109364225F
:1007180011921295139308A800F048FA0F23039337
:10072800049505944FF4805306930794032103A876
:1007380000F074FC15B030BD003802400070004075
:1007480008B500F0A7F8FFF7B3FFFFF7EBFEFFF7D8
:100758003DFFFEE782B0002100910B4B5A6C42F43A
:1007680080425A645A6C02F480420092009A0191C5
:100778001A6C42F080521A641B6C03F08053019388
:10078800019B02B0704700BF0038024002680E4B60
:100798009A4200D0704700B583B00021019103F55B
:1007A80074435A6C42F400325A645B6C03F40033AD
:1007B8000193019B0A46192000F0AAF8192000F0BD
:1007C800DBF803B05DF804FB004401407047FEE726
:1007D800FEE7FEE7FEE770477047704708B500F090
:1007E80073F808BD08B5012000F0D2F908BD000073
:1007F80008B5024800F0E9FC08BD00BF2C00002045
:100808000F49D1F8883043F47003C1F888300D4B94
:100818001A6842F001021A60002098601A6822F0F3
:10082800847222F480321A60074A5A601A6822F4E5
:1008380080221A60D8604FF000638B60704700BF59
:1008480000ED00E0003802401030002410B50446E6
:100858000E4B18784FF47A73B3FBF0F30C4A106818
:10086800B0FBF3F000F096F868B90F2C01D901201D
:100878000AE0002221464FF0FF3000F049F8034B10
:100888005C60002000E0012010BD00BF04000020D3
:100898000000002008B50B4B1A6842F400721A6079
:1008A8001A6842F480621A601A6842F480721A6008
:1008B800032000F01BF80020FFF7C8FFFFF74AFFEE
:1008C800002008BD003C0240034A1168034B1B7816
:1008D8000B441360704700BF6C0000200400002028
:1008E800014B1868704700BF6C000020074AD368A6
:1008F80023F4E0631B041B0C000200F4E0601843BF
:1009080040F0BF6040F40030D060704700ED00E078
:1009180030B4174BDB68C3F30223C3F10704042C7C
:1009280028BF04241D1D062D18D9033B4FF0FF35A1
:1009380005FA04F421EA0401994005FA03F322EACE
:100948000303194300280BDB0901C9B200F1604019
:1009580000F5614080F8001330BC70470023E5E7DC
:1009680000F00F000901C9B2024B1954F4E700BFA7
:1009780000ED00E014ED00E0002807DB00F01F02A6
:10098800400901239340024A42F82030704700BFD3
:1009980000E100E00138B0F1807F0AD2064B5860D0
:1009A800064AF02182F823100020986007221A6076
:1009B80070470120704700BF10E000E000ED00E044
:1009C80000230F2B00F2C580F0B482B039E0042276
:1009D80000E00022B2403A4302345E4E46F824203A
:1009E8005D4A1468EA4302EA04064F6817F4803F38
:1009F80001D045EA0406584C2660646802EA0406F9
:100A08004F6817F4003F01D045EA0406524C66606F
:100A1800A46802EA04064F6817F4801F01D045EA6B
:100A280004064D4CA660E46822404E6816F4001F88
:100A380001D045EA0402484CE26001330F2B00F272
:100A4800858001229A400C6804EA0205AA42F4D182
:100A58004C68022C01D0122C10D1DE08083650F850
:100A680026C003F00704A7000F24BC402CEA040C9E
:100A78000C69BC4044EA0C0440F8264004685F0056
:100A88000326BE40F64306EA040C4C6804F003044F
:100A9800BC4044EA0C0404604C6804F1FF3CBCF11F
:100AA800010F03D9112C01D0122C10D1846806EA49
:100AB800040CCC68BC4044EA0C048460446824EA12
:100AC80002024C68C4F300149C4014434460C2689A
:100AD80016408A68BA403243C2604A6812F0805FA2
:100AE800ABD0002201921D4A546C44F480445464F3
:100AF800526C02F480420192019A9C08A61C154A85
:100B080052F8267003F0030296000F22B24027EA3B
:100B18000207134A90423FF45CAF02F580629042AC
:100B28000ED002F5806290420CD002F580629042AD
:100B38000AD002F5806290423FF449AF072249E7A4
:100B4800012247E7022245E7032243E702B0F0BC4F
:100B58007047704700380140003C014000380240AF
:100B6800000002400369194201D1002070470120AA
:100B7800704712B909048161704781617047436900
:100B880031EA030301D0816170470904816170472C
:100B980008B5054B5B69034200D108BD024B58619B
:100BA800FFF72AFDF9E700BF003C0140002800F0EC
:100BB800BB8170B582B00446036813F0010F3BD0C7
:100BC800A74B9B6803F00C03042B2CD0A44B9B6809
:100BD80003F00C03082B21D06368B3F5803F4FD096
:100BE800B3F5A02F52D09E4B1A6822F480321A60B7
:100BF8001A6822F480221A606368002B50D0FFF72D
:100C08006FFE0546964B1B6813F4003F14D1FFF79F
:100C180067FE401B6428F5D903208AE1904B5B6886
:100C280013F4800FD8D08E4B1B6813F4003F03D009
:100C38006368002B00F07A81236813F0020F55D007
:100C4800874B9B6813F00C0F3ED0854B9B6803F0D5
:100C58000C03082B33D0E368002B68D0814B0122AA
:100C68001A60FFF73DFE05467D4B1B6813F0020F27
:100C780054D1FFF735FE401B0228F5D9032058E16F
:100C8800774A136843F480331360B5E7744B1A68E6
:100C980042F480221A601A6842F480321A60ABE784
:100CA800FFF71EFE05466E4B1B6813F4003FC3D0CA
:100CB800FFF716FE401B6428F5D9032039E1684B7D
:100CC8005B6813F4800FC6D1654B1B6813F0020FE5
:100CD80004D0E368012B01D001202AE1604A13689F
:100CE80023F0F803216943EAC1031360236813F072
:100CF800080F40D0636963B35B4B01221A60FFF7AA
:100D0800EFFD0546564B5B6F13F0020F33D1FFF72B
:100D1800E7FD401B0228F5D903200AE1504A136871
:100D280023F0F803216943EAC1031360DEE74D4B62
:100D380000221A60FFF7D4FD0546494B1B6813F0E3
:100D4800020FD3D0FFF7CCFD401B0228F5D90320B2
:100D5800EFE0454B00221A60FFF7C2FD0546404B05
:100D68005B6F13F0020F06D0FFF7BAFD401B022895
:100D7800F5D90320DDE0236813F0040F79D0384B50
:100D88001B6C13F0805F33D100230193344B1A6C32
:100D980042F080521A641B6C03F080530193019B4C
:100DA8000125324B1B6813F4807F23D0A368012BE5
:100DB80034D0052B38D02A4B1A6F22F001021A675B
:100DC8001A6F22F004021A67A368002B36D0FFF7C7
:100DD80087FD0646224B1B6F13F0020F48D1FFF721
:100DE8007FFD801B41F288339842F3D90320A0E0AD
:100DF8000025D6E71D4A136843F480731360FFF794
:100E08006FFD0646194B1B6813F4807FCED1FFF7A0
:100E180067FD801B0228F5D903208AE0104A136F6A
:100E280043F001031367CFE70D4B1A6F42F004023A
:100E38001A671A6F42F001021A67C5E7FFF750FDFB
:100E48000646074B1B6F13F0020F11D0FFF748FD42
:100E5800801B41F288339842F3D9032069E000BF30
:100E68000038024000004742800E474200700040B0
:100E7800E5B9A369002B5BD0304A926802F00C02F6
:100E8800082A58D0022B17D02D4B00221A60FFF7E2
:100E980027FD0446294B1B6813F0007F42D0FFF75B
:100EA8001FFD001B0228F5D9032042E0234A136CDA
:100EB80023F080531364DCE7214B00221A60FFF70C
:100EC8000FFD05461D4B1B6813F0007F06D0FFF78A
:100ED80007FD401B0228F5D903202AE0E369226AAE
:100EE8001343626A43EA8213A26A5208013A43EA48
:100EF8000243E26A43EA0263104A5360104B01223C
:100F08001A60FFF7EDFC04460C4B1B6813F0007FDA
:100F180006D1FFF7E5FC001B0228F5D9032008E0FD
:100F2800002006E0002004E001207047012000E0D6
:100F3800002002B070BD0120FBE700BF003802406E
:100F480060004742324B9B6803F00C03042B5CD0D3
:100F5800082B01D02F4870472DE9F04B2C4B5A68CD
:100F680002F03F025B6813F4800F2BD0284B5B68BC
:100F7800C3F388131E4600275C010025E41A65EBBD
:100F88000705A90141EA9461A001001B61EB050175
:100F9800CB0043EA5073C400A01943EB07014B028E
:100FA80043EAD0534402204619460023FFF710F9BC
:100FB800174B5B68C3F3014301335B00B0FBF3F0ED
:100FC800BDE8F08B124B5B68C3F388131E460027FD
:100FD8005C010025E41A65EB0705A90141EA946163
:100FE800A001001B61EB0501CB0043EA5073C4006C
:100FF800A01943EB07018B0243EA90538402204671
:1010080019460023FFF7E4F8D2E70348704700BF0A
:10101800003802400024F40000127A00002800F092
:101028009D8070B504464F4B1B6803F00F038B423D
:1010380009D2CBB24B4A1370136803F00F038B42EB
:1010480001D0012070BD236813F0020F17D013F0F0
:10105800040F04D0444A936843F4E0539360236830
:1010680013F0080F04D0404A936843F46043936038
:101078003D4A936823F0F003A068034393600D464C
:10108800236813F0010F32D06368012B21D09A1E18
:10109800012A25D9344A126812F0020F60D0324969
:1010A8008A6822F0030213438B60FFF719FC064697
:1010B8002D4B9B6803F00C036268B3EB820F16D0CC
:1010C800FFF70EFC801B41F288339842F0D90320C9
:1010D800B8E7254A126812F4003FE0D10120B1E7D1
:1010E800214A126812F0007FD9D10120AAE71D4BCE
:1010F8001B6803F00F03AB4209D9EAB2194B1A7007
:101108001B6803F00F03AB4201D001209AE7236864
:1011180013F0040F06D0144A936823F4E053E168EF
:101128000B439360236813F0080F07D00E4A9368A7
:1011380023F46043216943EAC1039360FFF702FF88
:10114800094B9B68C3F30313084AD35CD840084B88
:1011580018600020FFF77AFB002073E70120704732
:1011680001206FE7003C024000380240901400085C
:10117800000000200268D36843F00103D3600268CE
:10118800936803F00703062B03D0136843F00103A9
:101198001360002070470268D36823F00103D3600E
:1011A8000368196A41F21112114208D1196A40F212
:1011B8004442114203D11A6822F001021A60002049
:1011C8007047704770477047704710B5044603680A
:1011D8001A6912F0020F11D0DA6812F0020F0DD05E
:1011E8006FF002021A610123037703689B6913F009
:1011F800030F70D0FFF7E6FF0023237723681A69EF
:1012080012F0040F12D0DA6812F0040F0ED06FF04B
:1012180004021A610223237723689B6913F4407F31
:101228005FD02046FFF7CEFF0023237723681A6993
:1012380012F0080F12D0DA6812F0080F0ED06FF013
:1012480008021A61042323772368DB6913F0030F6C
:101258004ED02046FFF7B6FF0023237723681A698C
:1012680012F0100F12D0DA6812F0100F0ED06FF0D3
:1012780010021A61082323772368DB6913F4407F7F
:101288003DD02046FFF79EFF0023237723681A6985
:1012980012F0010F03D0DA6812F0010F36D123687B
:1012A8001A6912F0800F03D0DA6812F0800F34D177
:1012B80023681A6912F0400F03D0DA6812F0400F61
:1012C80032D123681A6912F0200F03D0DA6812F0BD
:1012D800200F30D110BDFFF774FF2046FFF773FFD2
:1012E8008AE72046FFF76DFF2046FFF76CFF9BE774
:1012F8002046FFF766FF2046FFF765FFACE720466C
:10130800FFF75FFF2046FFF75EFFBDE76FF00102C2
:101318001A612046FFF788F9C1E76FF080021A6169
:10132800204600F077F8C3E76FF040021A612046C4
:10133800FFF74AFFC5E76FF020021A61204600F068
:1013480068F8C7E70368254A90420ED0B0F1804F8D
:101358000BD0A2F57C42904207D002F58062904201
:1013680003D002F58062904203D123F070034A68EB
:1013780013431A4A90421AD0B0F1804F17D0A2F501
:101388007C42904213D002F5806290420FD002F561
:10139800806290420BD002F59A32904207D002F553
:1013A8008062904203D002F58062904203D123F418
:1013B8004073CA68134323F080034A6913430360E8
:1013C8008B68C3620B688362044B984202D0012386
:1013D800436170470B690363F9E700BF00000140F0
:1013E800A8B110B5044690F83D305BB1022384F8EB
:1013F8003D30211D2068FFF7A5FF012384F83D300B
:10140800002010BD80F83C30FFF7C0F9EEE701205E
:10141800704770477047000070B50D4E0D4CA41B07
:10142800A4100025A54209D10B4E0C4C00F020F861
:10143800A41BA4100025A54205D170BD56F825307F
:1014480098470135EEE756F8253098470135F2E719
:10145800B0140008B0140008B0140008B414000850
:1014680002440346934200D1704703F8011BF9E791
:10147800F8B500BFF8BC08BC9E467047F8B500BF79
:08148800F8BC08BC9E46704749
:101490000000000000000000010203040607080924
:0814A00000000000010203043A
:0814A80060EDFF7F0100000070
:0414B000BD01000872
:0414B4009901000892
:0C14B8000024F4000100000010000000FF
:04000005080004D912
:00000001FF
